:020000040000FA
:10000000830101308A000E29F300030E8301F400FE
:100010000A08F5008A010B1183120313A00F11289F
:10002000A10AA30F1428A40AA60F1728A70AB40F21
:100030001A28B50AC80F1D28C90AD10F2028D20ACC
:100040008316D90F2428DA0ADB0F2728DC0AEC0FE5
:100050002A28ED0AEE0F2D28EF0A83120317A10FAD
:100060003228A20AA60F3528A70AA80F3828A90AFD
:10007000AB0F3B28AC0AC10F3E28C20AC50F41286E
:10008000C60AC90F4428CA0A75088A00740E83007C
:10009000F30E730E09008B138B1B4B2877088A0015
:1000A00076088200831203130612FE20F60B5528F1
:1000B0000608F0390338860086165E288612F61682
:1000C000FE20F60B6028861665288612FE2086160E
:1000D00069288612FE2006106D2886166F28861263
:1000E000FE202830EB200C30EB200630EB20831272
:1000F000031306120130EB20F616FE20F60B7D28C6
:10010000FE2883120313061240307718F6071430C6
:10011000F718F607F617EC288312031306169C202F
:100120008B17FF3903190800F60000308A00EC2015
:10013000F90F8F28FA0A8F288B137A088A0079081A
:1001400082001030F6002730F700C620FC08031D9F
:10015000AA280121E830F6000330F700C620FC0889
:10016000031DB32801216430F600F701C620FC0806
:10017000031DBB2801210A30F600F701C620FC0848
:10018000031DC328012130307907E828FC08031D2E
:10019000FC03FB01FB0A7608F9027708031C770FC2
:1001A000FA020318CA287708FA077608F90703182D
:1001B000FA0A7B03031D7D1408000F39F600303066
:1001C000F6073A307602031CE7280730F607760870
:1001D000831203130616F600F801760E0F39F700A6
:1001E000831203130608F039770486008616F82870
:1001F0008612781BFE2878177608EE28F80BFE2862
:100200000800031DFC03F600031D7D1430307D182B
:10021000F60720307D1CF6077608E82820308B0092
:100220008312031300308500003086000030870001
:100230000F308316810006309F00FF308500C030EC
:100240008600DF3087008313203084008001840A19
:10025000841F262984168001840AF0300402031DBD
:100260002B298317103084008001840A7030040227
:10027000031D3429903084008001840AF030040288
:10028000031D3C29C03083120313CB000230D4007D
:10029000522081010B118B17831203130518542967
:1002A000A001A101221061298312031322186129E0
:1002B00001302102031C612938302002031C61290E
:1002C00022148312031385186929A301A401A51020
:1002D000762983120313A518762901302402031C02
:1002E000762938302302031C7629A51483120313C0
:1002F00005197E29A601A701A8128B2983120313D1
:10030000A81A8B2901302702031C8B2938302602BA
:10031000031C8B29A8160030831203130718013819
:10032000871802380719043887190838A900F60118
:1003300083165D08031DA02957088312AA00E62929
:10034000F60A83165D087602031DAA295708831250
:10035000AB00E629F60A83165D087602031DB42970
:1003600057088312AC00E629F60A83165D08760268
:10037000031DBE2957088312AD00E629F60A83162D
:100380005D087602031DC82957088312AE00E629CE
:10039000F60A83165D087602031DD22957088312D8
:1003A000AF00E629F60A83165D087602031DDC29F4
:1003B00057088312B000E629F60A83165D08760214
:1003C000031DE62957088312B100E629831603139B
:1003D000CE1CED298312B201F629831203133318C0
:1003E000F62983164E1CF6298312B20A83160313CC
:1003F0004E1CFD2983123314002A83120313331079
:1004000036180A2A83164E1C0A2A8312B401B50133
:10041000B614A81783120313B61C182A0930350224
:10042000031D142A28303402031C182AB610A813FE
:10043000831603134E1C1F2A83123614222A83129A
:10044000031336100B302A0283120313031D2A2ACA
:10045000A2142B2AA210F60183166808031D342A61
:1004600057088312B7007A2AF60A831668087602BC
:10047000031D3E2A57088312AA007A2AF60A831619
:1004800068087602031D482A57088312B8007A2AA2
:10049000F60A831668087602031D522A570883124B
:1004A000AA007A2AF60A831668087602031D5C2AD7
:1004B00057088312B9007A2AF60A8316680876026A
:1004C000031D662A57088312AA007A2AF60A8316A1
:1004D00068087602031D702A57088312BA007A2A28
:1004E000F60A831668087602031D7A2A57088312D3
:1004F000AA007A2AF601831603136908031D842AC9
:1005000057088312BB00D12AF60A83160313690821
:100510007602031D8F2A57088312AA00D12AF60AF1
:100520008316031369087602031D9A2A570883125B
:10053000BC00D12AF60A8316031369087602031D4C
:10054000A52A57088312AA00D12AF60A8316031394
:1005500069087602031DB02A57088312BD00D12A0C
:10056000F60A8316031369087602031DBB2A57088F
:100570008312AA00D12AF60A8316031369087602A9
:10058000031DC62A57088312BE00D12AF60A831615
:10059000031369087602031DD12A57088312AA00A3
:1005A000D12AF601831603136A08031DDB2A5708B4
:1005B0008312BF00282BF60A831603136A087602FB
:1005C000031DE62A57088312AA00282BF60A831671
:1005D00003136A087602031DF12A57088312C0002C
:1005E000282BF60A831603136A087602031DFC2AD9
:1005F00057088312AA00282BF60A831603136A08E9
:100600007602031D072B57088312C100282BF60A18
:10061000831603136A087602031D122B57088312F0
:10062000AA00282BF60A831603136A087602031D14
:100630001D2B57088312C200282BF60A83160313BA
:100640006A087602031D282B57088312AA00282B5C
:1006500083120313A21C302BC71F302B2215332B00
:10066000831203132211471F392BA21C392BA21509
:100670003C2B83120313A211C71E422BA21C422B38
:100680002216452B83120313221209302B028312E8
:100690000313031C4D2B031D4F2BA216502BA2122C
:1006A000471C582BA21E582BC71C582B22175B2BFC
:1006B000831203132213F60183166B08031D642BA8
:1006C00057088312C300AA2BF60A83166B0876021A
:1006D000031D6E2B57088312AA00AA2BF60A831655
:1006E0006B087602031D782B57088312C400AA2BCF
:1006F000F60A83166B087602031D822B57088312B5
:10070000AA00AA2BF60A83166B087602031D8C2B0F
:1007100057088312C500AA2BF60A83166B087602C7
:10072000031D962B57088312AA00AA2BF60A8316DC
:100730006B087602031DA02B57088312C600AA2B54
:10074000F60A83166B087602031DAA2B570883123C
:10075000AA00AA2B0B30831203132E028312031359
:10076000031DB42BC714B52BC7104A18BF2B831613
:100770004E1CBF2B8312C801C901CA144B1383122C
:100780000313CA1CCD2B7A304902031DC92B12302A
:100790004802031CCD2BCA104B17831603134E1CA3
:1007A000D42B83124A14D72B831203134A108316B7
:1007B00025088312500283120313031DE12BCC146E
:1007C000E22BCC10831626088312500283120313E7
:1007D000031DEC2B4C15ED2B4C11831627088312AF
:1007E0005B0283120313031DF72BCC15F82BCC11DE
:1007F0008316280883125B0283120313031D022C45
:100800004C16032C4C12F60183163408031D0E2CD3
:10081000831203171D080313CD00402CF60A83161C
:1008200034087602031D182C83123908CD00402CA1
:10083000F60A831634087602031D222C83123B0825
:10084000CD00402CF60A831634087602031D2C2CAA
:1008500083123D08CD00402CF60A83163408760238
:10086000031D362C83124008CD00402CF60A831657
:1008700034087602031D402C83124208CD00402C20
:10088000F601831603133408031D4A2C8312400813
:10089000CE00602CF60A8316031334087602031D7B
:1008A000552C83124208CE00602CF60A83160313DF
:1008B00034087602031D602C83124308CE00602C9E
:1008C000F601831603133408031D6C2C83120317DF
:1008D0001D080313CF00A32CF60A83160313340854
:1008E0007602031D772C83123908CF00A32CF60A59
:1008F0008316031334087602031D822C83123B08EF
:10090000CF00A32CF60A8316031334087602031DC6
:100910008D2C83124008CF00A32CF60A83160313F4
:1009200034087602031D982C83124208CF00A32CB2
:10093000F60A8316031334087602031DA32C8312D0
:100940004308CF00A32CF601831203135708031D9D
:10095000AC2C4D08D000C02CF60A831203135708A4
:100960007602031DB62C4E08D000C02CF60A831266
:10097000031357087602031DC02C4F08D000C02C6B
:100980007A30831203135202031DC82C1230510215
:10099000031CD52C7A30D2021230D102031CD203B0
:1009A000D31AD42CD316D52CD31283120313550883
:1009B0008316340283120313031CE02CD410E12CA1
:1009C000D414F6015708031DE82C0530D500082D76
:1009D000F60A57087602031DF02C0330D500082DC7
:1009E000F60A57087602031DF82C0530D500082DAD
:1009F000F60A57087602031D002D0330D500082D96
:100A0000F60A57087602031D082D0030D500082D80
:100A100000308312031322190138221A0238A21956
:100A20000438221B0838D600E130F6001A30F700EF
:100A30005608F6070318F70A00308A004B20831285
:100A40000313D7008B178A110A12D31E312DD41C21
:100A5000312DD31F312D83164D18312D831253178D
:100A6000342D831203135313F60183163408031D28
:100A70003D2D83123808D8006F2DF60A83163408EE
:100A80007602031D472D83123A08D8006F2DF60A0F
:100A9000831634087602031D512D83123C08D800BA
:100AA0006F2DF60A831634087602031D5B2D831220
:100AB0003E08D8006F2DF60A831634087602031D0F
:100AC000652D83124108D8006F2DF60A831634086D
:100AD0007602031D6F2D83124408D8006F2DF60196
:100AE000831603133408031D792D83124108D9009E
:100AF0008F2DF60A8316031334087602031D842D06
:100B000083124408D9008F2DF60A83160313340884
:100B10007602031D8F2D00308312D9008F2DF60130
:100B2000831603133408031D992D83123808DA0045
:100B3000C52DF60A8316031334087602031DA42D6F
:100B400083123A08DA00C52DF60A83160313340817
:100B50007602031DAF2D83123C08DA00C52DF60A7C
:100B60008316031334087602031DBA2D831241083D
:100B7000DA00C52DF60A8316031334087602031D26
:100B8000C52D83124408DA00C52DF6018312031324
:100B90005708031DCE2D5808DB00E22DF60A8312FC
:100BA000031357087602031DD82D5908DB00E22DE8
:100BB000F60A8312031357087602031DE22D5A0822
:100BC000DB00E22D831203135C18F92D83162B1F13
:100BD000F92D0030F6000130F70000308A00812046
:100BE000F130F9001A30FA0000308A008C208A11A6
:100BF0000A12831603132B1F002E83125C14032E7C
:100C0000831203135C105D18182E83162B1D182EEB
:100C10000030F6000230F70000308A0081200630F4
:100C2000F9001B30FA0000308A008C208A110A1269
:100C3000831603132B1D1F2E83125D14222E831285
:100C400003135D105E18372E8316AB1D372E003050
:100C5000F6000230F70000308A0081201B30F900D6
:100C60001B30FA0000308A008C208A110A12831689
:100C70000313AB1D3E2E83125E14412E8312031309
:100C80005E105F18562E8316AB1D562E0030F600F0
:100C90000130F70000308A0081203030F9001B302D
:100CA000FA0000308A008C208A110A12831603137E
:100CB000AB1D5D2E83125F14602E831203135F1031
:100CC0006018752E8316231C752E0030F600013037
:100CD000F70000308A0081204530F9001B30FA000F
:100CE00000308A008C208A110A1283160313231CF9
:100CF0007C2E831260147F2E831203136010611800
:100D0000942E8316231C942E0030F6000230F70038
:100D100000308A0081205A30F9001B30FA00003080
:100D20008A008C208A110A1283160313231C9B2E1F
:100D3000831261149E2E8312031361106218B32E66
:100D40008316A41FB32E0030F6000130F7000030E8
:100D50008A0081206F30F9001B30FA0000308A00D1
:100D60008C208A110A1283160313A41FBA2E831231
:100D70006214BD2E8312031362106318D22E8316E1
:100D8000A41FD22E0030F6000230F70000308A0097
:100D900081208430F9001B30FA0000308A008C205A
:100DA0008A110A1283160313A41FD92E8312631407
:100DB000DC2E8312031363106418F12E8316AA1C11
:100DC000F12E0030F6000130F70000308A0081205B
:100DD0009930F9001B30FA0000308A008C208A110B
:100DE0000A1283160313AA1CF82E83126414FB2E16
:100DF0008312031364106518102F8316AA1C102F7A
:100E00000030F6000230F70000308A008120AE305A
:100E1000F9001B30FA0000308A008C208A110A1277
:100E200083160313AA1C172F831265141A2F83121B
:100E30000313651066182F2F8316AA1D2F2F00305D
:100E4000F6000130F70000308A008120C330F9003D
:100E50001B30FA0000308A008C208A110A12831697
:100E60000313AA1D362F83126614392F831203131E
:100E7000661067184E2F8316AA1D4E2F0030F600FD
:100E80000230F70000308A008120D830F9001B3092
:100E9000FA0000308A008C208A110A12831603138C
:100EA000AA1D552F83126714582F8312031367103E
:100EB00068186D2F8316AA1E6D2F0030F6000130C2
:100EC000F70000308A008120ED30F9001B30FA0075
:100ED00000308A008C208A110A1283160313AA1E7E
:100EE000742F83126814772F831203136810691804
:100EF0008C2F8316AA1E8C2F0030F6000230F700CC
:100F000000308A0081200230F9001C30FA000030E5
:100F10008A008C208A110A1283160313AA1E932FAB
:100F200083126914962F8312031369106A18AB2F6A
:100F300083164E1DAB2F0030F6000330F700003053
:100F40008A0081201730F9001C30FA0000308A0036
:100F50008C208A110A12831603134E1DB22F83129E
:100F60006A14B52F831203136A106B18CA2F8316E5
:100F7000CE1DCA2F0030F6000030F70000308A0086
:100F800081202C30F9001C30FA0000308A008C20BF
:100F90008A110A1283160313CE1DD12F83126B14EC
:100FA000D42F831203136B106C18E92F83162B1D9B
:100FB000E92F0030F6000130F70000308A00812070
:100FC0004130F9001C30FA0000308A008C208A1170
:100FD0000A12831603132B1DF02F83126C14F32FA8
:100FE000831203136C108A15002800000000000013
:100FF00000000000000000000000000000000000F1
:101000006D1814284C1C14280030F6000030F7002E
:1010100000308A0081205630F9001C30FA00003080
:101020008A008C208A150A12831203134C1C1A287A
:101030006D141D28831203136D106E1831284C1C7B
:1010400031280030F6000130F70000308A0081209E
:101050006B30F9001C30FA0000308A008C208A15B1
:101060000A12831203134C1C37286E143A28831279
:1010700003136E106F184E284C1C4E280030F600DB
:101080000230F70000308A0081208030F9001C30E7
:10109000FA0000308A008C208A150A12831203138A
:1010A0004C1C54286F145728831203136F107018A8
:1010B0006B284C1C6B280030F6000330F700003022
:1010C0008A0081209530F9001C30FA0000308A0037
:1010D0008C208A150A12831203134C1C7128701479
:1010E000722870107118882883160313A31E88288D
:1010F0000030F6000130F70000308A008120AA306D
:10110000F9001C30FA0000308A008C208A150A127F
:1011100083160313A31E8E2871148F287110721862
:10112000A52883160313231EA5280030F6000130DE
:10113000F70000308A008120BF30F9001C30FA002F
:1011400000308A008C208A150A1283160313231E8E
:10115000AB287214AC287210831603132018C2280F
:10116000A31DC2280030F6000130F70000308A00CD
:101170008120D430F9001C30FA0000308A008C2025
:101180008A150A1283160313A31DC8282014CB281E
:101190008316031320102118DF28231DDF280030B9
:1011A000F6000130F70000308A008120E930F900B4
:1011B0001C30FA0000308A008C208A150A1283162F
:1011C0000313231DE5282114E82883160313211097
:1011D0002218FC28A31CFC280030F6000030F70081
:1011E00000308A008120FE30F9001C30FA00003007
:1011F0008A008C208A150A1283160313A31C022965
:10120000221405298316031322108312221A172988
:10121000A219172922191729221B1729471917293B
:101220000317B41917298316031323131A298316D6
:10123000031323178312CC1C22298316A41E2229F0
:101240002414252983160313241083124C1D2E29E0
:101250008316A41E2E298312CC173129831203135F
:10126000CC13CC1D3D298316A41E3D2983120317E0
:1012700014183D2903134C174029831203134C13F0
:101280004C1E4C298316A41E4C29831203171418D4
:101290004C290313CC164F2983120313CC12F601E9
:1012A00083162908031D57290C30A5006029F60A6A
:1012B000831629087602031D60290D30A5006029D8
:1012C000F601831603132908031D69290D30A600B2
:1012D0007329F60A8316031329087602031D73295E
:1012E0000C30A6007329F601831603132908031D89
:1012F0007C290C30A7008629F60A831603132908D7
:101300007602031D86290D30A7008629F601831673
:1013100003132908031D8F290D30A8009929F60A07
:101320008316031329087602031D99290C30A8009F
:101330009929003083160313A4180138A90003303B
:10134000340283160313031CA9290319A92924169F
:10135000AA2924120230340283160313031CB42971
:101360000319B429A415B529A411241ABF2983127D
:10137000221ABF2983162419BF29A410C229831653
:101380000313A4148312A21DCA298316A41DCA29FB
:101390002415CD298316031324118312221DD72966
:1013A0008316241FD729A31FD729A417DA29831648
:1013B0000313A4130030340283160313031DE22920
:1013C0002417E32924138312221DED2983162A1CD6
:1013D000ED29A31FED29AA14F02983160313AA10DF
:1013E0000130340283160313031DF8292A14F92946
:1013F0002A108312221D032A83162A1D032AA31FE3
:10140000032AAA15062A83160313AA1102303402EE
:1014100083160313031D0E2A2A150F2A2A1183127D
:10142000221D192A83162A1E192AA31F192AAA1651
:101430001C2A83160313AA120330340283160313E3
:10144000031D242A2A16252A2A128312221D2F2A36
:1014500083162A1F2F2AA31F2F2AAA17322A831680
:101460000313AA130430340283160313031D3A2A0C
:101470002A173B2A2A13AA1B432A311B432A361850
:10148000432AAB11462A83160313AB158312221D80
:10149000502A83162B1C502AA31F502AAB14532A00
:1014A00083160313AB100530340283160313031D98
:1014B0005B2A2B145C2A2B10AB18642AB619642AF9
:1014C000361A642A2B11672A831603132B152C183E
:1014D0007B2A2B1F7B2A0030F6000230F7000030F9
:1014E0008A0081201330F9001D30FA0000308A0094
:1014F0008C208A150A12831603132B1F812A2C14A1
:10150000842A831603132C108312A21D8E2A83169D
:101510002B1E8E2AA31F8E2AAB16912A8316031325
:10152000AB120530340283160313031D992A2B16C0
:101530009A2A2B12AB1AA02A361BA02A2B13A32AF5
:10154000831603132B178312A21DAD2A8316AB1F1C
:10155000AD2AA31FAD2A2314B02A83160313231028
:101560000030340283160313031DB82AAB17B92ABF
:10157000AB132D18CD2AA31CCD2A0030F600023063
:10158000F70000308A0081202830F9001D30FA0071
:1015900000308A008C208A150A1283160313A31CBC
:1015A000D32A2D14D62A831603132D102E18EA2AB7
:1015B000A31CEA2A0030F6000330F70000308A004E
:1015C00081203D30F9001D30FA0000308A008C2067
:1015D0008A150A1283160313A31CF02A2E14F32A69
:1015E000831603132E108312A21FFB2A8316231FB8
:1015F000FB2AA314FE2A83160313A3108312A21F2F
:10160000062B221E062B8316A316092B8316031303
:10161000A3128312A21F112BA21D112B83162316B6
:10162000142B8316031323128312A21F1C2B221DBB
:101630001C2B8316A3151F2B83160313A3118312D0
:10164000A21F272B221F272B831623152A2B831635
:10165000031323112F183E2BB11C3E2B0030F60034
:101660000130F70000308A0081205230F9001D302F
:10167000FA0000308A008C208A150A1283160313A0
:10168000B11C442B2F14472B831603132F10301833
:101690005B2BB11C5B2B0030F6000230F7000030F2
:1016A0008A0081206730F9001D30FA0000308A007E
:1016B0008C208A150A1283160313B11C612B301477
:1016C000642B8316031330108312A21D6E2B831616
:1016D000311C6E2BA31F6E2BB114712B83160313B9
:1016E000B1100130340283160313031D792B31141A
:1016F0007A2B311032188E2BB11D8E2B0030F60054
:101700000130F70000308A0081207C30F9001D3064
:10171000FA0000308A008C208A150A1283160313FF
:10172000B11D942B3214972B8316031332103318E8
:10173000AB2BB11DAB2B0030F6000230F7000030B0
:101740008A0081209130F9001D30FA0000308A00B3
:101750008C208A150A1283160313B11DB12B331482
:10176000B42B8316031333108312A21DBE2B8316D2
:10177000311DBE2BA31FBE2BB115C12B8316031326
:10178000B1110230340283160313031DC92B311526
:10179000CA2B31118312A21FD02B8316B401E02B68
:1017A00083160313311EE02B3518E02B35148312FA
:1017B000A81ADD2B8316B40AE02B83160313B40397
:1017C00083160313311AE52B35108312531BED2BAF
:1017D000D319ED2B83163112F02B83160313311618
:1017E0008312281FF92B8316A31FF92B8312D315FD
:1017F000FC2B83120313D311281A022CA819022CD4
:101800002813052C831203132817A21D0E2C8316F0
:10181000B11E0E2CA31F0E2C3117112C831603138F
:1018200031130330340283160313031D192CB11630
:101830001A2CB1128312221E242C8316B11F242CC1
:10184000A31F242C3614272C8316031336100030C4
:10185000340283160313031D2F2CB117302CB11340
:101860008312A21D3A2C8316B61C3A2CA31F3A2CC5
:10187000B6153D2C83160313B611043034028316BB
:101880000313031D452CB614462CB6108312221EDA
:10189000502C8316361D502CA31F502C3616532C5B
:1018A0008316031336120130340283160313031D0B
:1018B0005B2C36155C2C36118312221E662C831687
:1018C000B61E662CA31F662C3617692C83160313CD
:1018D00036130230340283160313031D712CB6161F
:1018E000722CB6123718862C241C862C1130F60068
:1018F0000130F70000308A008120A630F9001D3049
:10190000FA0000308A008C208A150A12831603130D
:10191000241C8C2C37148F2C831603133710381883
:10192000A42C8312CC1FA42C1130F6000130F70038
:1019300000308A008120A930F9001D30FA00003003
:101940008A008C208A150A1283120313CC1FAB2C39
:1019500083163814AE2C8316031338103918C32C91
:1019600083124C1FC32C1130F6000230F7000030F8
:101970008A008120AC30F9001D30FA0000308A0066
:101980008C208A150A12831203134C1FCA2C83164B
:101990003914CD2C8316031339103A18E22C831214
:1019A000CC1EE22C1130F6000230F70000308A0025
:1019B0008120AF30F9001D30FA0000308A008C2001
:1019C0008A150A1283120313CC1EE92C83163A14CB
:1019D000EC2C831603133A103B18002D441C002DE9
:1019E0000030F6000130F70000308A008120B2306C
:1019F000F9001D30FA0000308A008C208A150A1286
:101A000083160313441C062D3B14092D8316031360
:101A10003B103C181D2DC41C1D2D0030F60001305C
:101A2000F70000308A008120C730F9001D30FA002D
:101A300000308A008C208A150A1283160313C41CF6
:101A4000232D3C14262D831603133C103D183A2DEC
:101A5000C61C3A2D0030F6000230F70000308A0034
:101A60008120DC30F9001D30FA0000308A008C2023
:101A70008A150A1283160313C61C402D3D14432DEC
:101A8000831603133D103E18572D491D572D003066
:101A9000F6000230F70000308A008120F130F900B2
:101AA0001D30FA0000308A008C208A150A12831635
:101AB0000313491D5D2D3E14602D831603133E1044
:101AC0003F18742D491F742D0030F6000130F700C7
:101AD00000308A0081200630F9001E30FA00003004
:101AE0008A008C208A150A1283160313491F7A2D47
:101AF0003F147D2D831603133F104018912D461D72
:101B0000912D0030F6000230F70000308A0081206D
:101B10001B30F9001E30FA0000308A008C208A1534
:101B20000A1283160313461D972D40149A2D83160F
:101B3000031340104118AE2DC61DAE2D0030F60027
:101B40000230F70000308A0081203030F9001E306A
:101B5000FA0000308A008C208A150A1283160313BB
:101B6000C61DB42D4114B72D83160313411042181E
:101B7000CB2DC61FCB2D0030F6000130F700003012
:101B80008A0081204530F9001E30FA0000308A00BA
:101B90008C208A150A1283160313C61FD12D4214F6
:101BA000D42D8316031342104318E92D8312A81C69
:101BB000E92D0030F6000230F70000308A00812065
:101BC0005A30F9001E30FA0000308A008C208A1545
:101BD0000A1283120313A81CF02D83164314F32D4D
:101BE0008316031343100030340283160313031DBE
:101BF000FB2D4417FC2D44134518102E441D102EA8
:101C00000030F6000130F70000308A0081206F308C
:101C1000F9001E30FA0000308A008C208A150A1262
:101C200083160313441D162E4514192E8316031311
:101C30004510441F252EC41E252EA31F252E8312BA
:101C4000221F252E83164414282E831603134410B6
:101C5000441F342E441E342EA31F342E8312221F01
:101C6000342E8316C414372E83160313C410441F56
:101C7000432EC41D432EA31F432E8312221F432E27
:101C800083164415462E831603134411B61B562E95
:101C9000C41F562E461C562EA31F562E441F562ECA
:101CA0008312221F562E8316C614592E8316031331
:101CB000C6100130340283160313031D612E46172C
:101CC000622E4613B61F722EC41B722E461C722E35
:101CD000A31F722E441F722E8312221F722E831690
:101CE0004615752E831603134611B61F852EC41F85
:101CF000852E4618852EA31F852E441F852E831200
:101D0000221F852E8316C615882E83160313C6112F
:101D100047189C2E461E9C2E0030F6000230F7001D
:101D200000308A0081208430F9001E30FA00003033
:101D30008A008C208A150A1283160313461EA22ECF
:101D40004714A52E831603134710B61FB52EC41FC4
:101D5000B52E461CB52EA31FB52E441FB52E8312DB
:101D6000221FB52E83164616B82E8316031346126D
:101D70004818CC2E491CCC2E0030F6000130F7005C
:101D800000308A0081209930F9001E30FA000030BE
:101D90008A008C208A150A1283160313491CD22E3E
:101DA0004814D52E831603134810C61EE12EA31F18
:101DB000E12E461FE12E8312221FE12E8316C61745
:101DC000E42E83160313C613C61AF02E461FF02EF8
:101DD000A31FF02E8312221FF02E83164914F32E18
:101DE0008316031349104A18072FC91D072F003007
:101DF000F6000230F70000308A008120AE30F90092
:101E00001E30FA0000308A008C208A150A128316D0
:101E10000313C91D0D2F4A14102F831603134A10E4
:101E2000C91C1C2FA31F1C2F461F1C2F8312221FEF
:101E30001C2F831649151F2F831603134911C91828
:101E40002B2F461F2B2FA31F2B2F8312221F2B2F2D
:101E50008316C9152E2F83160313C91102303402BD
:101E600083160313031D362FC916372FC912491EB7
:101E7000432FA31F432FC91E432F8312221F432F1B
:101E800083164917462F831603134913491A522FF5
:101E9000C91E522FA31F522F8312221F522F8316A7
:101EA000C917552F83160313C9138312281C622FD9
:101EB0008316A31F622FC91E622F8312221F622F57
:101EC000A814652F83120313A8102818712F8316E6
:101ED000C91E712FA31F712F8312221F712F281566
:101EE000742F83120313281183164B18892FC91FCF
:101EF000892F0030F6000130F70000308A00812081
:101F0000C330F9001E30FA0000308A008C208A1598
:101F10000A1283160313C91F8F2F4B14922F831697
:101F200003134B104C18A72F8312281DA72F003026
:101F3000F6000230F70000308A008120D830F90026
:101F40001E30FA0000308A008C208A150A12831293
:101F50000313281DAE2F83164C14B12F83160313C1
:101F60004C108312D41CB82F221CB82F2816BB2F5C
:101F70008312031328125319C12FA81EC12FA815AD
:101F8000C42F83120313A811003083163402831266
:101F90000313031DCD2F5315CE2F5311A21BD52F85
:101FA000281FD82F83164D14D82F831603134D10D6
:101FB00083120313A81BE22F83164F18E22F4F142E
:101FC000CE14EA2F83160313CE108312A81FEA2F14
:101FD00083164F108A110A16002800000000000026
:101FE00000000000000000000000000000000000F1
:101FF00000000000000000000000000000000000E1
:102000008316031350181A28CE1D1A280530F6001F
:102010000030F70000308A008120831203174C083B
:10202000F900FA017D100330FC0000308A00B32073
:102030008A110A1683160313CE1D20285014232854
:1020400083160313501051183B28CE1D3B28063031
:10205000F6000030F70000308A0081208312031759
:102060004D08F900FA017D100330FC0000308A00B1
:10207000B3208A110A1683160313CE1D412851146A
:10208000442883160313511052185B28CE1D5B2879
:102090001230F6000030F70000308A0081208312F1
:1020A00003171908F90000308A00790EDD2079083D
:1020B000DD208A110A1683160313CE1D61285214DF
:1020C0006428831603135210A31F6A284E1E6A2821
:1020D000CE156D2883160313CE118312221A792888
:1020E000A2197928221979284719792883164E12BE
:1020F0007C28831603134E1653189028CE1E902862
:102100000030F6000030F70000308A008120ED300A
:10211000F9001E30FA0000308A008C208A110A165D
:1021200083160313CE1E962853149928831603137F
:1021300053105418B128CE1EB1280F30F6000030CD
:10214000F70000308A008120831203132B08F90066
:10215000FA017D100330FC0000308A00B3208A11A0
:102160000A1683160313CE1EB7285414BA288316F2
:10217000031354105518D228CE1ED2281030F60062
:102180000030F70000308A00812083120317150801
:10219000F900FA017D100330FC0000308A00B32002
:1021A0008A110A1683160313CE1ED8285514DB286D
:1021B0008316031355105618F328CE1EF32811303A
:1021C000F6000030F70000308A00812083120317E8
:1021D0001708F900FA017D100330FC0000308A0076
:1021E000B3208A110A1683160313CE1EF92856143B
:1021F000FC28831603135610A31F02294E1F022921
:10220000CE16052983160313CE12F6015808031DB6
:102210000C295708D7001629F60A58087602031D1C
:102220001629831229088316D70016290030831631
:102230000313CE1B0138D8005708831229028316D6
:10224000031303192529CE172629CE134E1C2D2939
:10225000D901DA01831253143C2983120313531C4E
:102260003C29003083165A02031C3C299C30590239
:10227000031C3C298312531083120313531846295D
:102280008316DB01DC018312D3105529831203135B
:10229000D3185529003083165C02031C55294E3093
:1022A0005B02031C55298312D314F6018316031312
:1022B0005E08031D5E296430DD006A29F60A831674
:1022C00003135E087602031D6A29831232088316FF
:1022D000DD006A29003083120313D31801388316F6
:1022E000DE005F1C8B2983120317431A8B290B30E6
:1022F000F6000230F70000308A00812083120313B9
:102300002B08F900FA017D100330FC0000308A0030
:10231000B3208A110A1683120317431E93298316CA
:1023200003135F149629831603135F10601CB029F2
:1023300083120317C31AB0290C30F6000230F700DD
:1023400000308A008120831203171508F900FA0172
:102350007D100330FC0000308A00B3208A110A1679
:1023600083120317C31EB829831603136014BB29F5
:10237000831603136010611CD52983120317C31B36
:10238000D5290D30F6000230F70000308A00812098
:10239000831203171708F900FA017D100330FC00BF
:1023A00000308A00B3208A110A1683120317C31F54
:1023B000DD29831603136114E029831603136110CA
:1023C000621CF929831203174418F9290D30F6000D
:1023D0000230F70000308A008120831203171F08A3
:1023E000F90000308A00790EDD207908DD208A119D
:1023F0000A1683120317441C012A8316031362145E
:10240000042A831603136210631C1E2A8312031707
:10241000C4181E2A0F30F6000230F70000308A0080
:102420008120831203175308F900FA017D1003304D
:10243000FC0000308A00B3208A110A1683120317A9
:10244000C41C262A831603136314292A8316031334
:102450006310641C432A831203174419432A103063
:10246000F6000230F70000308A0081208312031743
:102470001908F900FA017D100330FC0000308A00D1
:10248000B3208A110A1683120317441D4B2A8316A0
:10249000031364144E2A831603136410651C682A00
:1024A00083120317C41B682A1130F6000230F700AC
:1024B00000308A008120831203171B08F900FA01FB
:1024C0007D100330FC0000308A00B3208A110A1608
:1024D00083120317C41F702A831603136514732A0B
:1024E000831603136510661C8D2A83120317C41903
:1024F0008D2A1230F6000230F70000308A00812069
:10250000831203171D08F900FA017D100330FC0047
:1025100000308A00B3208A110A1683120317C41DE3
:10252000952A831603136614982A831603136610DC
:102530008312531EA12A8316A31FA12A83124B14B0
:10254000A42A831203134B10221AAE2AA219AE2A10
:102550002219AE2A221BAE2A5312B12A8312031368
:10256000531683166718C82A83120317431CC82AF8
:102570000030F6000130F70000308A008120023080
:10258000F9001F30FA0000308A008C208A110A16E8
:1025900083120317431CD02A831603136714D32A0C
:1025A00083160313671008305D02E80010305D02E7
:1025B000E90018305D02EA0020305D02EB00A31B49
:1025C000E62AEC01ED018312D313F52A83120313DB
:1025D000D31BF52AB73083166D02031CF52A1B3076
:1025E0006C02031CF52A8312D31783120313D41E23
:1025F000FF2A8316EE01EF01831254140E2B83126F
:102600000313541C0E2B0C3083166F02031C0E2B6D
:1026100035306E02031C0E2B8312541083120313E9
:10262000A81A1C2B22181C2B54191C2BD4191C2B38
:10263000541A1C2BD4121F2B83120313D4165418B4
:10264000282B03171018282B1014031354172F2BA3
:10265000831203135413541C2F2B031710108316CB
:102660000313A31F3B2B8312031711183B2B1114C9
:1026700003135415442B8312031354118316A31B05
:10268000442B83120317111083160313311E502B92
:10269000831203171218502B12140313D415592B3D
:1026A00083120313D4118316311A592B8312031783
:1026B000121083120313D41C642B03171318642BFA
:1026C0001314031354166B2B831203135412D418D0
:1026D0006B2B0317131083120313541F7E2B8316C7
:1026E000A31F7E2B8312221B7E2B47197E2B0317E1
:1026F000B4197E2B83160313A416812B83160313A0
:10270000A4128312221A882BA219882BD4138B2B84
:1027100083120313D417D41F922BD418922B0317B0
:102720001414952B831203171410F6011608031DB9
:102730009E2B03132C0803179500A82BF60A1608E6
:102740007602031DA82B03132B0803179500A82B53
:102750000E30831203132C0283120317031DB22BB6
:102760009414B32B94100030941801389600F6019D
:102770001808031DC02B03132D0803179700CA2B3D
:10278000F60A18087602031DCA2B03132C08031738
:102790009700CA2B0E30831203132D0283120317E6
:1027A000031DD42B1415D52B141100301419013826
:1027B0009800F6011A08031DE22B031330080317D3
:1027C0009900EA2BF60A1A087602031DEA2B530831
:1027D0009900EA2B0E308312031330028312031781
:1027E000031DF42B9415F52B941100309419013826
:1027F0009A00F6011C08031D022C0313310803176D
:102800009B000C2CF60A1C087602031D0C2C0313EB
:10281000300803179B000C2C0E3083120313310277
:1028200083120317031D162C1416172C14120030D4
:10283000141A01389C00F6011E08031D242C0313F2
:10284000370803179D002E2CF60A1E087602031D7A
:102850002E2C0313310803179D002E2C0E308312EB
:102860000313370283120317031D382C9416392CD7
:1028700094120030941A01389E00F6012008031DBE
:10288000462C03132E0803179F00502CF60A20082D
:102890007602031D502C03132D0803179F00502CA4
:1028A0000E30831203132E0283120317031D5A2CBA
:1028B00014175B2C14130030141B0138A0000313F1
:1028C0002518702C8316311A702C8312A21B702CC1
:1028D000A81A702CA518702C2218702CA511732C16
:1028E00083120313A5150317941F7B2CA101A201CA
:1028F000031325158A2C83120313251D8A2CF4300B
:1029000003172202031C8A2C24302102031C8A2C68
:1029100003132511831203134B1C962C0317231842
:10292000962C2314831603134E159E2C8316031323
:102930004E1183124B189E2C03172310831203137E
:102940004B1EA52C0317A401AE2C831203172518C8
:10295000AE2C03134B1DAE2C0317A40A83120313D2
:102960004B1DB52C03172514B82C83120317251003
:102970005B302702031DBE2C8E302602031CCC2C9C
:102980005B30A7028E30A602031CA7030313CB18EB
:10299000CB2CCB14CC2CCB1083120313CB1CD42CFC
:1029A000CB19D42C4B15D72C831203134B11C830E1
:1029B0000317240283120313031CE02CCB15E12C14
:1029C000CB11CB1BE92C0317A801A9010313CB12D0
:1029D000F82C83120313CB1AF82C0C30031729029E
:1029E000031CF82C35302802031CF82C0313CB16DB
:1029F00083120313CB178316CE1F042D83122519C0
:102A0000042D83164E14072D831603134E108312C4
:102A1000CB1E112D03172A18112D2A140313251468
:102A2000182D831203132510CB1A182D03172A1003
:102A300083120313A51D212D0317AB01AC019417BD
:102A40002E2D83120317941F2E2DF4302C02031CFD
:102A50002E2D24302B02031C2E2D941383120317CA
:102A60002D18452D0313251E452D0030F60002308C
:102A7000F70000308A0081201730F9001F30FA007B
:102A800000308A008C208A110A1683120313251E37
:102A90004C2D03172D144F2D831203172D10831661
:102AA0000313C618622D4619622DC619622D461AE7
:102AB000622D441F622DA31F622D8312221F622DDF
:102AC0002516652D83120313251203172E186C2D5E
:102AD00083160313C6126F2D83160313C6168312B3
:102AE0000317AE18772D8316031349127A2D831618
:102AF00003134916831203172E19822D831603130D
:102B0000C413852D83160313C4172C30F6001F3011
:102B1000F700831203171908F6070318F70A0030A5
:102B20008A004B2083120317AE008B178A110A16F6
:102B30002F189E2D83160313C910A12D831603137E
:102B4000C91483120317AF18A82D03132810AA2D38
:102B50000313281403172F19B12D83160313B6136B
:102B6000B42D83160313B6172C30F6001F30F70070
:102B7000831203171B08F6070318F70A00308A00B0
:102B80004B2083120317AF008B178A110A163018D7
:102B9000CD2D83160313C412D02D83160313C41630
:102BA00083120317B018D82D831603134412DB2D9C
:102BB000831603134416831203173019E32D83166B
:102BC0000313C411E62D83160313C41583120317D0
:102BD000B019EE2D831603134610F12D831603133F
:102BE00046143C30F6001F30F700831203175308D9
:102BF000F6070318F70A00308A004B2083120317E8
:102C0000B0008B178A110A16031325180B2ECB1947
:102C10000B2E4C100E2E831203134C148316CE1C55
:102C20001A2E8312A51E1A2E03174B1C1A2E0313DD
:102C3000A2171D2E83120313A2134B1F282EA51EAD
:102C4000282E03174B1C282E83160313A3172B2E95
:102C500083160313A3130930831232028312031362
:102C6000031C342E2517352E2513A51B3B2E251F9F
:102C70003E2EA5163E2E83120313A51283120313B4
:102C8000A81F492E03173118492E31140313A51715
:102C9000502E83120313A513A81B502E03173110B7
:102CA000053083120317530283120313031C5A2E99
:102CB000031D5C2E47145D2E471003173218732E28
:102CC0000313C71D732E0030F6000130F7000030EB
:102CD0008A0081204C30F9001F30FA0000308A0051
:102CE0008C208A110A1683120313C71D7A2E03172C
:102CF00032147D2E8312031732100313A21F842E69
:102D0000471E842EC715872E83120313C71103177E
:102D100033188D2E0313C7138F2E0313C7170317F2
:102D2000B318952E03134713972E03134717031752
:102D300033199D2E0313C7129F2E0313C71661303C
:102D4000F6001F30F70003171908F6070318F70AF3
:102D500000308A004B2083120317B3008B178A11AF
:102D60000A1603134718BB2EC71CBB2E0317C41E1D
:102D7000BB2EB414BE2E83120317B410341EC82EFB
:102D800083160313A31FC82E831203173414CB2EEC
:102D90008312031734103518DF2E441FDF2E003046
:102DA000F6000230F70000308A0081207130F9000F
:102DB0001F30FA0000308A008C208A110A16831214
:102DC0000317441FE52E3514E82E83120317351020
:102DD0003618002F441F002F1330F6000230F70082
:102DE00000308A008120831203171D08F900FA01C0
:102DF0007D100330FC0000308A00B3208A110A16CF
:102E000083120317441F062F3614092F831203174A
:102E10003610371C222F83160313CD18222F0A30A9
:102E2000F6000130F70000308A008120831203137E
:102E30002B08F90000308A00790EDD207908DD20AA
:102E40008A110A1683160313CD1C2A2F8312031727
:102E500037142D2F8312031737103818432F83167A
:102E60000313CD1F432F0030F6000030F700003071
:102E70008A0081208630F9001F30FA0000308A0075
:102E80008C208A110A1683160313CD1F4B2F831231
:102E9000031738144E2F8312031738103918642F74
:102EA00083160313CD1C642F0030F6000130F700A9
:102EB00000308A0081209B30F9001F30FA0000307A
:102EC0008A008C208A110A1683160313CD1C6C2FDE
:102ED0008312031739146F2F8312031739103A1C0A
:102EE000892F83160313CD18892F0C30F60001307B
:102EF000F70000308A008120831203171508F900BB
:102F0000FA017D140330FC0000308A00B3208A11DE
:102F10000A1683160313CD1C912F831203173A143C
:102F2000942F831203173A103B1CAC2F4B19AC2F74
:102F30000D30F6000130F70000308A008120831246
:102F400003171708F900FA017D140330FC00003064
:102F50008A00B3208A110A16831203174B1DB22F61
:102F60003B14B52F831203173B103C1CCC2FCB18FE
:102F7000CC2F0D30F6000130F70000308A008120A0
:102F8000831203171F08F90000308A00790EDD2034
:102F90007908DD208A110A1683120317CB1CD22F61
:102FA0003C14D52F831203173C103D1CEE2F8316C3
:102FB0000313CD18EE2F0E30F6000130F70000306D
:102FC0008A008120831203175308F90000308A0019
:102FD000790EDD207908DD208A110A168316031385
:102FE000CD1CF62F831203173D14F92F83120317FC
:102FF0003D108A15002800000000000000000000BD
:103000003E181428C31C14280030F6000230F700C4
:1030100000308A008120B030F9001F30FA00003003
:103020008A008C208A150A1683120317C31C1A28DB
:103030003E141D28831203173E100730031332027B
:1030400083160313031D26284D1527284D118312BF
:10305000A81B2F2883164D1D2F28CD153228831627
:103060000313CD1106308312320283160313031D9E
:103070003B284D163C284D128312A81B442883166A
:103080004D1E4428CD14472883160313CD108312F8
:1030900003173F185D28431D5D280030F6000330FC
:1030A000F70000308A008120C530F9001F30FA0097
:1030B00000308A008C208A150A1683120317431DDC
:1030C00063283F146628831203173F1040187C289A
:1030D00083160313CD1E7C280030F6000230F70063
:1030E00000308A008120DA30F9001F30FA00003009
:1030F0008A008C208A150A1683160313CD1E842895
:103100008312031740148728831203174010831675
:103110000313CD1C8F284D1B8F28CD1692288316A4
:103120000313CD12CD1D9C2883120317C101C201C8
:10313000831603134D17AD28831603134D1FAD28B7
:103140003D30831203174202031CAD2809304102AF
:10315000031CAD28831603134D1383120317C319E1
:10316000BB2883160313CD19BB2883120317B41B86
:10317000BB284310BE28831203174314C319CA285F
:1031800083160313CD19CA2883120317B41BCA2848
:10319000C310CD2883120317C314C319D92883166B
:1031A0000313CD19D92883120317B41BD92843124E
:1031B000DC28831203174316C319E8288316031368
:1031C000CD19E82883120317B41BE828C312EB2893
:1031D00083120317C316C319F72883160313CD19D7
:1031E000F72883120317B41BF7284313FA28831216
:1031F00003174317C319062983160313CD1906298C
:1032000083120317B41B06294410092983120317DC
:103210004414C319152983160313CD1915298312D4
:103220000317B41B1529C410182983120317C414DB
:10323000C319242983160313CD19242983120317D4
:10324000B41B242944112729831203174415C718D6
:103250003329471C3F290313D4183F290317C501FD
:10326000C601C71444160130831203174602031D1A
:103270003B2938304502031C3F29C71044128312F2
:103280000313D41C46290317471449298312031733
:10329000471006301B0283120317031C5129031D1C
:1032A0005329C4165429C412C3195C29B41B5C29C0
:1032B000441B5C29C4135F2983120317C417341CF1
:1032C000662948186629481444176C298312031785
:1032D000441334186C2948108312031734197429C5
:1032E000B41C7429B415772983120317B411341D43
:1032F0007E29B41C7E2903134715812983120313E9
:1033000047110E302B0283120317031D8929341530
:103310008A2934110313471992290317B4199229E2
:10332000341295298312031734160313221B9F2985
:103330000317B4199F29831603134E13A22983166A
:1033400003134E1783122519AB290317B41AAB299F
:1033500003138712AE298312031387160317341F32
:10336000B529C901CA01B416C22983120317B41EB4
:10337000C229F4304A02031CC22924304902031C2A
:10338000C229B41283160313CD18CE29CD19CE2924
:1033900083120317B41BCE293413D12983120317C8
:1033A0003417341BD82903132519D8294B12DB29CC
:1033B000831203134B160317441EE4290313221F21
:1033C000E4290317C315E72983120317C311031355
:1033D0004719F0290317B419F02903134712F329E9
:1033E0008312031347168316CD19002ACD18002A1D
:1033F00083120317B41B002A83160313CD13032A69
:1034000083160313CD17CD190D2ACD180D2A83125B
:103410000317B41B0D2A4311102A831203174315F7
:103420000313221A222AA219222A221B222A221933
:10343000222A0317B419222A03134719222A031731
:103440004B10252A831203174B14C3192B2AB41BC4
:103450002B2AC4112E2A83120317C41583160313B3
:10346000CE1C3C2A831203174B183C2A0313A51EBB
:103470003C2A0317B4173F2A83120317B413F6012B
:103480004E08031D462A1708CC004E2AF60A4E089D
:103490007602031D4E2A1508CC004E2AF60183122F
:1034A00003174E08031D572A1F08CD00612AF60A8C
:1034B000831203174E087602031D612A1708CD00F8
:1034C000612A003083120313471901380317CE0015
:1034D0004F1C7C2ACB187C2A0A30F6000130F700FA
:1034E00000308A008120EF30F9001F30FA000030F0
:1034F0008A008C208A150A1683120317CB1C822A95
:103500004F14852A831203174F1083160313CD1807
:10351000902A831203175018902A5014CB149A2A19
:1035200083120317CB1083160313CD1C9A2A831220
:103530000317501083120317431BA32A5118A32A01
:103540005114C317A92A83120317C313431FA92AAF
:10355000511083120317CB18B22A5218B22A5214F0
:103560004B15B82A831203174B11CB1CB82A5210E3
:10357000F601831203175408031DC32A03132F08EF
:103580000317D300CF2AF60A8312031754087602D2
:10359000031DCF2A03132E080317D300CF2A0E30A2
:1035A000831203132F0283120317031DD92ACB158D
:1035B000DA2ACB110030CB190138D4008A110A1253
:1035C0004C29043400340134043402340434043407
:1035D000043403340434043404340434043404342C
:1035E000043441346C346C34613472346D34653479
:1035F00020342034533469346E34633472346F347D
:103600003A342034203420342034003441346C34B3
:103610006C342E342034453466346634723461346C
:103620007A3469346F346E3465343A34203420345B
:1036300020342034003441346C346C3461347234BE
:103640006D346534203420342034203452346534D1
:10365000743465343A342034203420342034003437
:1036600041346C346C34613472346D3465342034DC
:1036700050346F34743465346E347A3461343A348F
:1036800020342034203420340034523469346334FC
:103690002E342034203443346934723463346F342C
:1036A0006C346134723465343A342034203420343C
:1036B0002034003454347234613473342E34203462
:1036C00043346934723463346F346C34613472342B
:1036D00065343A34203420342034203400345434D7
:1036E0006F346E3469342034503472346F3476342D
:1036F00065346E34693465346E342E343A34203493
:1037000020342034203400345234693463342E346D
:103710002034543472346134743474346134203459
:103720006E342E3432343A34203420342034203471
:1037300000345234693463342E34203454347234B7
:10374000613474347434613420346E342E34333440
:103750003A34203420342034203400345234693454
:1037600063342E34203454347234613474347434F9
:10377000613420346E342E3434343A3420342034DE
:103780002034203400345234693463342E342034ED
:1037900054347234613474347434613420346E348B
:1037A0002E3435343A34203420342034203400345C
:1037B0005234693463342E342034543472346134D6
:1037C00074347434613420346E342E3436343A34E4
:1037D00020342034203420340034523469346334AB
:1037E0002E3420345434723461347434743461347B
:1037F00020346E342E3437343A342034203420349C
:10380000203400345234693463342E342034543438
:103810007234613474347434613420346E342E3430
:1038200038343A3420342034203420340034703496
:10383000613467342D342034203420342A342A343F
:103840002A342A342A34203420342034203470346A
:10385000613467342B340034523465347434653445
:103860003A342034203420342034413470347034DD
:1038700061347234613474346F343A342034203417
:10388000003441346C346C34613472342E3420345E
:10389000423461347434743465347234693461345C
:1038A0003A342034203420342034003443346F340C
:1038B000723470346F3420344E3461347A34693465
:1038C0006F346E3461346C3465342034563456347D
:1038D000463420340034433465346E3474347234E6
:1038E0006F34203454344C34433420344134623403
:1038F000723475347A347A346F342034203400349E
:10390000533469347334743465346D346134203421
:103910004D3469342E3443346F346E342E342034B5
:10392000563431342E343034003442347934203437
:1039300054346F347034703469342034473469340B
:103940007534733465347034703465342034203405
:1039500020340034203420345234693473347034C9
:103960006F347334743461342034523469346E34B7
:10397000763469346F3420342034203400342034D9
:1039800052346934733470346F3473347434613442
:10399000203453346134743465346C346C34693499
:1039A00074346534203400342034203420345234CC
:1039B0006934733470346F34733474346134203444
:1039C0004D346134733474346534723420342034AB
:1039D00000345234693473342E3420345334743404
:1039E000613474346F342034433469347234633452
:1039F0006F346C34613472346534003420342034D4
:103A000020342034203452346934633465347A34B9
:103A100069346F346E3465342034203420342034DB
:103A20002034203400342034203420342034203416
:103A300020342034203420342034203420342034E6
:103A400020342034203420342034203420340034F6
:103A500020342034203420342034203420342034C6
:103A600020342034203420342034203420342034B6
:103A700020342034203420340034203420342034C6
:103A80002034203420342034203420342034203496
:103A90002034203420342034203420342034203486
:103AA00020340034533463346F34723472342E341F
:103AB000203450346F347234743461346E3474345E
:103AC00065343A34203420342034203400345234E5
:103AD000693474346134723464346F342034203483
:103AE0003234303420344B346D3420343A34203482
:103AF0002034203420340034523469347434613436
:103B0000723464346F34203420343434303420340C
:103B10004B346D3420343A34203420342034203473
:103B200000345234693474346134723464346F3420
:103B300020342B342D343834303420344B346D342D
:103B40003A3420342034203420340034453458347E
:103B5000003449344E340034453458340034493448
:103B60004E340034463475346E347A342E34203476
:103B700020344E346F3472346D3461346C346534B7
:103B800020343A34203449344E342034003446341E
:103B900075346E347A342E342034203453347034F7
:103BA00065346334693461346C3465343A342034B8
:103BB00049344E342034003449346E3474342E3455
:103BC000203443346934723463342B3444346F34D6
:103BD0007234733420343A34203449344E3420342F
:103BE000003454346F346E346F34203432344434FF
:103BF0006F342D344E3464342F344C346B342034D1
:103C00003A34203449344E34203400345434693446
:103C10006D346534723420342034203444346F34AD
:103C20007234733461346C3465343A34203449343A
:103C30004E342034003449346E3474342E342034FD
:103C400043346934723463342B344C346B342F3442
:103C50004E3464343A34203449344E342034003401
:103C600049346E3474342E34203444346F34723416
:103C700073342B344C346B342F344E3464343A3434
:103C8000203449344E342034003454346F346E348C
:103C90006F3420342034203444346F34723473341D
:103CA00061346C34653420343A34203449344E3431
:103CB00020340034543469346D3465347234203423
:103CC000323444346F342D344E3464342F344C3415
:103CD0006B343A34203449344E3420340034463482
:103CE00075346E347A342E3420344134673465347C
:103CF00076346F346C34613474346F343A34203435
:103D000049344E342034003449346E3474342E3403
:103D1000433469342B3444346F342B344C346B3497
:103D20002F344E3464343A34203449344E34203401
:103D3000003454346F346E346F34203420342034E3
:103D400044346F347234733461346C3465342034E9
:103D50003A342034453458342034003454346F34E9
:103D60006E346F342034323444346F342D344E3456
:103D700064342F344C346B3420343A34203445349A
:103D8000583420340034543469346D34653472341A
:103D900020342034203444346F347234733461342A
:103DA0006C3465343A34203445345834203400348B
:103DB000543469346D3465347234203432344434CC
:103DC0006F342D344E3464342F344C346B343A34E5
:103DD00020344534583420340034203420344334E3
:103DE0006F34643469346334653420345234653458
:103DF000743465343A342034203420342034203470
:103E00002034003420342034203420342034203432
:103E10002034203420342034203420342034203402
:103E200020342034203420342034203400344934E9
:103E30006E3474346534723463346F346E346E347B
:103E40006534733473342E34203420343A342034BF
:103E500045345834203400340134053403340734F5
:103E600000340434023406340034003400340034A6
:103E700000340034003400340134093402340A348C
:103E800004340C3400340034003400340034003482
:103E900000340034003400342034543465346E343B
:103EA000733469346F346E346534203420344234D2
:103EB0006134743474346534723469346134203458
:103EC0000034043402340234023402340234023442
:103ED0000234023401340434043404340434043429
:103EE000043456346F346C347434203452346934AE
:103EF0006C346534763461347434693420343A3443
:103F00002034313420342E342034003444346534A9
:103F100063346F346434693466342E34203474343A
:103F20006F346E346934203443344334493452346A
:103F300020342034003443346F3464342E34353428
:103F400054346F346E3469343D342034203420349A
:103F500020342034203420342034203420340034E1
:103F600043342E3436342F34383454346F346E3472
:103F700069343D342034203420342034203420343B
:103F800020342034203420340034203420342034B1
:103F90002034203420342034203420342034203481
:103FA0002034203420342034203420342034203471
:103FB0002034003420342034203420342034203481
:103FC0002034203420342034203420342034203451
:103FD0002034203420342034203420340034203461
:023FE0000034AB
:084000000000010000000100B6
:02400E00723FFF
:00000001FF
